:020000040000FA
:020000000528D1
:040002000034003492
:08000800052821006B3099006E
:100010002100FF308C0000309500240011308C004E
:10002000220002309D00230011308C00220080301D
:1000300091002200C1309200220097012000980117
:1000400020008C0121000C1620009A019101013042
:100050009C0064309B0025008C3093000F30910091
:1000600020001C1592122100921640308B002000B7
:100070002000921263005B20382814309B00200877
:10008000A3009B032108A4009B0A2208A500A50B3E
:100090004728A40B4428A30B412808002008A300EC
:1000A0002108A4002208A500A50B5428A40B52285F
:1000B000A30B5028080021000C120C102000013066
:1000C000A0005A30A100FF30A2003D2021000C16F4
:1000D0000C1420000130A0002830A100FF30A20045
:0400E0004E200800A6
:020000040001F9
:02000E0084F973
:02001000FFDE11
:00000001FF
